:1000000050C068C067C066C065C064C063C062C0DD
:1000100061C060C05FC05EC05DC05CC05BC05AC0F4
:1000200059C058C057C057524F4E470A004F4B2136
:1000300020596F7527726520696E2E0A00456E740F
:10004000657220636F64652E0A00436869702068DA
:1000500061732073656C662D646573747275637467
:1000600065642120546568206E6F657A21212131F5
:100070000A002569207472696573206C6566742EA8
:100080000A0052656164792E0A0045464765666735
:1000900000202B2D2E303132333435363738396845
:1000A000000011241FBECFEDCDBF10E0A0E6B0E0F0
:1000B000ECE4F6E002C005900D92AE36B107D9F738
:1000C00010E0AEE6B0E001C01D92A437B107E1F741
:1000D00006D0BAC295CF5F9BFECF8CB10895AF9288
:1000E000BF92CF92DF92EF92FF921F93CF93DF9355
:1000F00082E090E093D2853A41F082E090E065EAB8
:1001000095D281E090E065E091D283E390E074D0F5
:1001100000D082E890E0EDB7FEB792838183FBD1F7
:100120000F900F9022E7A22E20E0B22E9DE3C92E61
:1001300090E0D92E86E2E82E80E0F82ECDE2D0E0E5
:1001400081E090E06BD2182F00D000D0EDB7FEB761
:10015000B282A182992787FD909594838383DBD116
:100160000F900F900F900F90112359F400D08AE454
:1001700090E0EDB7FEB792838183CDD10F900F90C1
:10018000FFCF00D0EDB7FEB7D282C182C4D10F90AD
:100190000F905F9BFECF9CB15F9BFECF8CB18233F3
:1001A00051F4943341F400D0EDB7FEB7D283C1834C
:1001B000B2D116E006C000D0EDB7FEB7F282E18200
:1001C000AAD10F900F9003C05F9BFECF8CB15F99B7
:1001D000FBCF115081E090E0612F28D2B1CF1F9367
:1001E000182F8A3011F48DE0FADF5D9BFECF1CB929
:1001F00080E090E01F91089528E12AB989B9892FFC
:10020000990F990B82B980E690E0909371008093EA
:1002100070000895ABE0B0E0EFE0F1E012C15C01E6
:100220004B017A01FC0117821682838181FD08C08F
:100230006FEF7FEFFEC042E050E0E40EF51E04C019
:100240003E010894611C711CF501D380F401D3FCBC
:100250008591D3FE81914F01882309F4E7C085324F
:1002600059F4D3FC6591D3FE61914F01653219F0C9
:10027000062F10E01AC085E290E029C0002309F49F
:10028000D5C081E990E0602F70E00ED1892B39F460
:10029000033211F4106103C00C3661F41068F401EC
:1002A000D3FC0591D3FE01914F0117FFE7CF002347
:1002B00009F4BCC08AE890E0602F70E0F5D0892B8B
:1002C00049F044E050E0E40EF51E8FE390E0B50104
:1002D000F6D0BACF033629F0033771F00335E1F4D5
:1002E0000AC087010E5F1F4FF70180819181B50120
:1002F000E6D07801A9CF1160F701C080D18003C09A
:1003000090E0B501DCD0F60110FD859110FF8191E0
:100310006F018823A9F78FCF043611F0093639F51C
:1003200017FF08C0F701208131814281538184E0A9
:1003300090E00AC0F701808191819C01442737FD3C
:100340004095542F82E090E0E80EF91E1F7E57FF83
:1003500008C050954095309521953F4F4F4F5F4FC6
:100360001064CA01B901A3012AE030E034C00037AB
:10037000A9F0013730F40835B1F00F3609F056C056
:1003800006C0053739F0083709F050C008C028E02A
:1003900030E00CC01F7E2AE030E008C0106114621B
:1003A00020E130E003C0146020E132E017FF08C014
:1003B000F701608171818281938144E050E008C03F
:1003C000F70180819181BC0180E090E042E050E043
:1003D000E40EF51EA301C2D0D82ED618012F10E0CE
:1003E00006FF04C08DE290E0B50169D004FF13C0A0
:1003F000FE01ED0DF11D8081803369F080E390E016
:10040000B5015DD002FF07C000721070C801885AA4
:100410009F4FB50154D0DA94F301ED0DF11D8081A9
:1004200090E0B5014CD0DD20B1F70ECFF50166812B
:100430007781CB012B96EEE020C02F923F924F9216
:100440005F926F927F928F929F92AF92BF92CF9264
:10045000DF92EF92FF920F931F93CF93DF93CDB76D
:10046000DEB7CA1BDB0B0FB6F894DEBF0FBECDBFE5
:1004700009942A88398848885F846E847D848C84B6
:100480009B84AA84B984C884DF80EE80FD800C81BF
:100490001B81AA81B981CE0FD11D0FB6F894DEBFA2
:1004A0000FBECDBFED010895FC010590061621F0A9
:1004B0000020D9F7C00108953197CF0108950F9317
:1004C0001F93CF93DF938C01EB018B8181FF1BC0C6
:1004D00082FF0DC02E813F818C819D8128173907B5
:1004E00064F4E881F9810193F983E88306C0E88523
:1004F000F985802F0995892B31F48E819F81019692
:100500009F838E8302C00FEF1FEFC801DF91CF9151
:100510001F910F910895A0E0B0E0E0E9F2E09DCFD7
:10052000FE01359661917191A0917000B0917100BA
:1005300013968C911397886013968C93809170001A
:1005400090917100AF0166DEE0917000F091710052
:100550002381277F23832096E2E09BCFFA01AA27FD
:10056000283061F1203191F1E8946F936E7F6E5FD6
:100570007F4F8F4F9F4FAF4FB1E040D0B4E03ED0A0
:10058000670F781F891F9A1FA11D680F791F8A1F87
:10059000911DA11D6A0F711D811D911DA11D22D0EC
:1005A00009F468943F91062E000C3019000C000CE1
:1005B0003019305D3193CEF6CF010895462F477044
:1005C000405D4193B3E00FD0C9F7F6CF462F4F708F
:1005D000405D4A3318F0495D31FD4052419302D0ED
:1005E000A9F7EACFB4E0A695979587957795679593
:1005F000BA95C9F700976105710508959B01AC0193
:100600000A2E06945795479537952795BA95C9F7B9
:10061000620F731F841F951FA01D0895E199FECFDF
:100620001FBA8EBBE09A99278DB30895262FE199C2
:10063000FECF1CBA1FBA8EBB2DBB0FB6F894E29A40
:0C064000E19A0FBE01960895F894FFCFD8
:0E064C000000000200000000EF0000000000AF
:00000001FF
